:020000040800F2
:10000000904B0020F9010008C9110008F110000808
:10001000C7110008850F000839150008000000000E
:10002000000000000000000000000000491200086D
:10003000DB10000800000000CB1100084D12000882
:10004000130200081302000813020008130200083C
:10005000130200081302000813020008130200082C
:10006000130200081302000813020008130200081C
:10007000130200081302000813020008130200080C
:1000800013020008130200081302000813020008FC
:10009000890F000813020008130200081302000869
:1000A00013020008391300081302000813020008A5
:1000B00013020008130200081302000813020008CC
:1000C00013020008130200081302000813020008BC
:1000D00013020008B5130008130200087514000885
:1000E000130200081302000813020008130200089C
:1000F00013020008130200080000000000000000C6
:1001000000000000000000000000000013020008D2
:10011000130200081302000813020008130200086B
:10012000130200081302000813020008130200085B
:100130001302000800000000000000001302000885
:10014000130200081302000813020008130200083B
:100150001302000813020008000000001302000848
:100160001302000813020008000000000000000055
:10017000000000000000000000000000000000007F
:100180000000000013020008130200081302000818
:10019000000000000000000000000000000000005F
:1001A000000000000000000000000000000000004F
:1001B0000000000000000000130200080000000022
:1001C000000000000000000000000000000000002F
:1001D0000000000000000000000000001302000802
:1001E000DFF810D000F08AFD00480047F544000811
:1001F000AFF30080904B0020064880470648004738
:10020000FEE7FEE7FEE7FEE7FEE7FEE7FEE7FEE7C6
:10021000FEE7FEE765120008E10100082DE9F05F46
:100220000546002092469B46884606468146402465
:100230001BE0284641464746224600F0C2FB534693
:100240005A46C01A914110D311461846224600F072
:10025000A9FB2D1A67EB01084F4622460120002119
:1002600000F0A0FB17EB00094E41201EA4F1010491
:10027000DFDC484631462A464346BDE8F09FA0F100
:100280004101192900D82030704740EA01039B073B
:1002900003D009E008C9121F08C0042AFAD203E0FB
:1002A00011F8013B00F8013B521EF9D27047D2B25F
:1002B00001E000F8012B491EFBD270470022F6E74F
:1002C00010B513460A4604461946FFF7F0FF2046CC
:1002D00010BD421C10F8011B0029FBD1801A704789
:1002E00010B5002200E0521C835C8C5CA34201D15B
:1002F000002BF8D1D8B2E1B2401A10BDCBB203E066
:100300000178994203D0401C521EF9D20020704758
:1003100030B504460020034600E05B1C934203D244
:10032000E05CCD5C401BF8D030BD30B50546002008
:10033000034600E05B1C934205D2EC5CC85C201ACB
:1003400001D1002CF6D130BD2DE9FF4F087883B0E4
:100350009946FF2805D0491C2D2804D000240020F0
:1003600008E000200BE00124F9E700EB800003EB3C
:100370004000491C0B78FF2BF7D104B14042002309
:100380000293147819461D462D2C01D02B2C04D134
:10039000521C2D2C13D000240294AA461478FF2C52
:1003A0000FD00A25A3FB057801FB05814FF0000C57
:1003B00003FB0C11521CE3194AEB0101EEE7012487
:1003C000EAE7814453EA010002D019F5C87F06DA52
:1003D00003980021C0E9001107B0BDE8F08F0025A7
:1003E000AE4E2F46DFF8B882184600F047FCCDE944
:1003F0000001B9F1000002DAC9F1000400E004468E
:100400000023A74A1AEB030B42EB045A12E0E00761
:1004100007D02A4633463846414600F0ECF90746F5
:1004200088462A4633461046194600F0E4F9054648
:100430000E466410002CEAD1DDE90001B9F1000F8D
:100440005A46534606DA00F0AAFB3A46434600F005
:10045000A6FB05E000F0CFF93A46434600F0CBF9A1
:10046000029A0AB181F00041039AC2E90001B3E7A0
:100470002DE9FF4F1F468DB0D7E901464FF0FF38F9
:100480002E2045464FF000090B90B9696D1C0E985F
:100490008847396A824688470028F6D1BAF1FF3F7B
:1004A0000AD024F4D064002E11DDBAF12B0F08D04D
:1004B000BAF12D0F0BD102E0404611B08DE744F4A4
:1004C0008064B9696D1C0E9888478246761E69461D
:1004D000600501D52D2000E02B208DF8000001F1F2
:1004E000010B0DF1200809E0B9696D1C0E988847D1
:1004F00082460F9844F40074761E0560002E02DDDB
:10050000BAF1300FF0D00B998A453ED144F0800407
:1005100006E00F99681CA9F1010944F40074086011
:10052000B9696D1C761E0E98884782463028F0D037
:100530002BE00B998A4505D1200603D444F08004B2
:10054000761E18E0504601F061F908B30DF1130171
:10055000761E44F400748B4508D2AAF130000BF8E3
:10056000010B200607D5A9F1010003E0200602D403
:1005700009F101008146A00502D50F99681C0860A9
:10058000B9696D1C0E9888478246002ED1DC53E075
:10059000002E51DDBAF1650F02D0BAF1450F4BD1F3
:1005A000A00549D5B9696D1C24F44074761E0E98D7
:1005B00088478246002E0CDD2B2804D0BAF12D0F7F
:1005C00007D144F48074B9696D1C0E98884782463F
:1005D000761EE00501D52D2100E02B2108F8011B36
:1005E000CDF82C8021E00DF12901761E44F4007431
:1005F00088450CD2AAF1300010F0FF0088F8000006
:1006000002D10B99884509D908F1010806E0E005F7
:1006100001D5244801E042F20F708146B9696D1C92
:100620000E98884782460F980560002E04DD5046DC
:1006300001F0ECF80028D6D1F9690E988847FF2020
:100640008BF8000088F800000020069007904B46C9
:100650006A4608A906A8FFF777FEA00502D46FF046
:1006600001002AE714F0240F0AD0E00714D1DDE9D5
:1006700006123868031D3B600068C0E900120BE0F9
:10068000DDE9060100F01EFB0146E00704D13868F1
:10069000021D3A600068016028460EE70000144021
:1006A0000000F03FF1D8FFFF2DE9FE4F804681EAC0
:1006B0000300C00F0C46009021F0004123F00045DC
:1006C000B8EB0200A94105D24046214690461C469F
:1006D0000B46024623F00040104347D0270DC7F3D6
:1006E0000A00C3F30A510290401A019040286BDAC5
:1006F000C3F3130040F4801B0098924620B10023FE
:10070000D2EB030A63EB0B0B01985946C0F1400290
:10071000504600F047F906460D4650465946019AA4
:1007200000F05FF910EB08006141002487EA1152E4
:1007300084EAE7731A4340D0009A62B3019A012A0F
:100740004FEA075215DC001B61EB02014FF000423B
:1007500002EA0752CDE90042001C41F58011324601
:100760002B4600F0CEF903B0BDE8F08F404621469D
:10077000F9E7001B61EB0201001C41F58013001832
:100780005B412018A2F5001747EB030140EAD57042
:10079000B6196D4111E06D084FEA360645EAC0759D
:1007A0004FEA0752001B61EB0201001C41F580116A
:1007B00049084FEA30000019514132462B4603B038
:1007C000BDE8F04F00F08EB90098012240000023F0
:1007D000D0EB020263EBE073009821464FEAE0742D
:1007E000B8EB000061EB0401E9E783F000435BE74D
:1007F00081F0004158E72DE9FE4F81EA030404F03F
:10080000004421F0004100944FF0000B23F000431E
:1008100050EA01045ED052EA03045BD0C3F30A54E9
:10082000C1F30A552C44A4F2F3340194A0FB025402
:10083000C1F3130141F48011C3F3130343F4801394
:1008400001FB024400FB034E840A970A44EA8154E8
:1008500047EA8357A4FB076802958D0A05FB0785C5
:100860004FEA932C04FB0C542705029D4FEA0658CF
:1008700047EA1637B5EB08056EEB070C870E920EAC
:1008800047EA811742EA8312A7FB0201B6EB0B018C
:1008900064EB00042B0D43EA0C335E1844EB1C5050
:1008A000DA465146E7FB0201C5F313044FEA0B3366
:1008B00043EA14534FEA0432019C43EA0603A4F1CD
:1008C0000C040294009CCDE900B400F01AF903B0C6
:1008D000BDE8F08F00200146F9E770B5C1F30A5278
:1008E00001F000450024C1F3130140F2FF3341F44D
:1008F00080119A4201DA002070BD40F233439A42DF
:10090000A2F2334203DC524200F05BF800E0904078
:100910002C43F1D0404270BD30B5041E71F100048B
:1009200004DB4FF00044404264EB0101141E73F1FC
:10093000000405DB1C464FF00043524263EB040306
:100940008B4208BF824230BD30B5041E71F10004F5
:1009500004DB4FF00044404264EB0101141E73F1CC
:10096000000405DB1C464FF00043524263EB0403D6
:10097000994208BF904230BD30B50B460146002079
:100980002022012409E021FA02F59D4205D303FA51
:1009900002F5491B04FA02F52844151EA2F10102D2
:1009A000F1DC30BD202A04DB203A00FA02F10020FD
:1009B00070479140C2F1200320FA03F3194390409D
:1009C0007047202A04DB203A21FA02F00021704708
:1009D00021FA02F3D040C2F12002914008431946A7
:1009E0007047202A06DBCB17203A41FA02F043EA8F
:1009F000E07306E041FA02F3D040C2F120029140D8
:100A0000084319467047426842B1016811F8013B3A
:100A100023B1521EC0E90012184670470121C1607F
:100A2000881E704742685AB1C368016843B9836839
:100A30008B4205D0491E521CC0E9001200207047AD
:100A40004FF0FF30704700000FB4002300B589B0AD
:100A50000CA900910B996FF00042CB601E4B0693DE
:100A60001E4B07930423CDE901321D4A089202462A
:100A70006B460020FFF7FCFC09B05DF814FB70B575
:100A800086B006464FF0FF300091CDE9010100200D
:100A900015460C4604903246694604A8FFF7D4FF79
:100AA00002460498211825B108B1084600E0204606
:100AB0002860049800280DD0002A02DD00988842A2
:100AC00008D0081B0094CDE901043246694604A809
:100AD000FFF7BAFF06B070BD070A0008250A000834
:100AE000290D000810B5141E73F1000408DA401C2B
:100AF00041F1000192185B411A4301D120F001003D
:100B000010BD2DE9F04D92469B4611B1B1FA81F22C
:100B100002E0B0FA80F220329046FFF743FF04462D
:100B20000F4640EA0A0041EA0B0153465A46084381
:100B300013D0114653EA010019D0C8F140025046C3
:100B4000FFF73FFF05460E46504659464246FFF71F
:100B500029FF084305D0012004E020463946BDE8BE
:100B6000F08D0020054346EAE0762C4337430A988F
:100B70006305E40AA0EB08000022FD0A44EA47549A
:100B80000A3002D500200146E9E701051019694144
:100B9000DDE9084500196941BDE8F04DA2E72DE9FE
:100BA000F04D81EA030404F0004B21F000451446A7
:100BB0004FF0000A23F0004150EA050220D054EA29
:100BC00001021DD0C5F30A570246C5F31303C1F352
:100BD0001300C1F30A5640F4801543F48013A7EBC9
:100BE0000608101BD64608F2FD3873EB050002D349
:100BF00008F1010801E092185B41B8F1000F03DA37
:100C000000200146BDE8F08D00204FF4801106461B
:100C100084460EE0171B73EB050705D3121B63EB2D
:100C2000050306434CEA010C49084FEA30009218CC
:100C30005B4150EA0107EDD152EA030012D082EA8B
:100C4000040083EA0501084305D0101BAB4106D21E
:100C50000122002306E000224FF0004302E06FF083
:100C6000010253101AEB06004CEB085110EB0A007E
:100C700041EB0B01BDE8F04DFFF734BF0EB540F27C
:100C8000334202920022CDE900221346FFF739FFDA
:100C900003B000BDC1F30A52C1F3130140F2FF33A8
:100CA00041F480119A4202DA00200146704740F276
:100CB00033439A42A2F2334202DC5242FFF781BE32
:100CC000FFF770BE01F0004330B421F0004150EA5C
:100CD000010206D00A0DA2F56072C1F31301002AC9
:100CE00002DC30BC00207047440F44EAC104C1005C
:100CF000E01830BC00EBC25000F01FB8064C074DA6
:100D000006E0E06840F0010394E8070098471034DB
:100D1000AC42F6D3FFF768FA0C6100082C610008BA
:100D200000487047C060000810B50446FFF7F8FFA0
:100D30000068005D00F0010010BD0029A8BF7047E9
:100D4000401C490008BF20F00100704710B4B0FA01
:100D500080FC00FA0CF050EA010404BF10BC70479C
:100D600049B1CCF1200421FA04F411FA0CF118BFB6
:100D7000012121430843A3EB0C01CB1D4FEA006185
:100D80004FEA102042BF002010BC704700EBC35058
:100D900010440029A4BF10BC7047401C490008BF84
:100DA00020F0010010BC704770B5734D7348744C4F
:100DB00069781A2914D2DFE801F00D9A9A9A14275B
:100DC0003E51646E78820D919A9A9A9EA8B2BCC6E2
:100DD000CCD2D89D082103F0BBF8202003F0B6FA4E
:100DE00085E0012000F07AF9297801EB410104EB5C
:100DF000C1010883002000F071F9297801EB41015D
:100E000004EBC10108857EE0012000F067F9297834
:100E100001EB410104EBC1014883002000F05EF9C1
:100E2000297801EB410104EBC101488575E000BF61
:100E300000F0CEF85BE0012000F050F9297801EBDA
:100E4000410104EBC1018883002000F047F92978B3
:100E500001EB410104EBC101888568E0012000F04D
:100E60003DF9297801EB410104EBC101C883002061
:100E700000F034F9297801EB410104EBC101C88588
:100E80005FE0012000F02AF9297801EB410104EB31
:100E9000C101C8845BE0012000F020F9297801EB52
:100EA000410104EBC101888457E0012000F016F9EC
:100EB000297801EB410104EBC101488453E0012092
:100EC00000F00CF9297801EB410104EBC101088421
:100ED000062000F07DF80C20687008E0082103F07F
:100EE00035F8254829782030405C03F093FA68787B
:100EF000401C687070BD012000F0F0F820800020D8
:100F000000F0ECF82082042092E7012000F0E6F8DF
:100F10006080002000F0E2F86082022088E7012073
:100F200000F0DCF8A080002000F0D8F8A0820120BA
:100F30007EE7012000F0D2F8E080002000F0CEF83B
:100F4000E082072074E7012000F0C8F8E081052066
:100F50006EE7012000F0C2F8A081032068E70120BD
:100F600000F0BCF86081002062E7012000F0B6F8D4
:100F7000208106205CE700000800002000000240FD
:100F80003C070020FEE7000010B5094C092120466F
:100F900002F010F901280AD10921204602F0DAF8FE
:100FA0002046BDE81040034A002102F05DB910BDA3
:100FB00000640040C8220020034610B5002002460D
:100FC00003E09C5C521C204480B28A42F9DB10BDD5
:100FD00070B50446104DC0074FF02001284602D0DE
:100FE00002F0B6FF01E002F0B1FFA0074FF01001E0
:100FF000284602D502F0ACFF01E002F0A7FF60072F
:101000004FF00801284603D5BDE8704002F0A0BFAC
:10101000BDE8704002F09ABF0004024070B5C160A4
:101020000546002614461046314600F0BDF8084338
:1010300007D14FF00040844202D2204600F0F0F881
:101040000446AE60C5E90046204670BD2DE9F0417A
:1010500004460E46D4E90110091A914200D20A460C
:10106000216817464A1E10400D1ABD4200D33D4666
:10107000E1682A4601443046FFF707F97A1B7019E8
:10108000E168FFF702F9A0683844A0603846BDE87F
:10109000F0812DE9F04104460E46D4E90101431ADE
:1010A0002168CB1A934200D21A4617464A1E1040B6
:1010B0000D1ABD4200D33D46E1682A460844314638
:1010C000FFF7E3F87A1B7119E068FFF7DEF8606854
:1010D000384460603846BDE8F0817047022803D28A
:1010E000024931F810007047002070477800002056
:1010F000FEE700002DE9F843054672B6284C20783B
:10110000E06005F59C70182229468046FFF7BDF87F
:10111000E068182200EB400005EBC00105F5A8705F
:1011200006461831FFF7B1F82078401C207020786F
:1011300000270C210C2807D1277001206060A068CF
:10114000401CA0600A2804D0A068092802DB677050
:1011500001E0A760617062B6124801230C22C0E969
:101160000086018105F5B4710E4603F073FA05F5AA
:10117000C071009700230C220F46304603F0ECF9B3
:10118000E068396800EB400005EB8000C0F88C1186
:101190007968C0F89011B968C0F89411BDE8F88377
:1011A00008000020A006002050EA010206D0421EDE
:1011B00041F1FF3302400B401A4302D00020C11717
:1011C00070470120FBE7FEE7704770471CB501211F
:1011D000114802F0A9F9684602F020FF01208DF8BD
:1011E000070000218DF804108DF8060038200B4C04
:1011F00000908DF805106946204602F019FF08217D
:10120000204602F0A3FE1021204602F09FFE20217E
:10121000204602F09BFE1CBD01003000000402408D
:1012200030B5044601250021FFF7BEFF084309D170
:1012300044B1E807844204D264084FEA4505FBD173
:10124000680830BD204630BD704700000448016882
:101250004268491C42F10002016042607047000090
:10126000380000201E4810B5016841F4700101608B
:10127000012002F09BF81B48016841F00101016068
:1012800001688907FCD5174908310A6822F0030272
:101290000A600A6812F00C0FFBD10268124B1A4068
:1012A00002604FF0804008600E491048091D086038
:1012B0000C48A030016801F4A0410160016841F4CC
:1012C0007021016007494FF41F000C3108600020B5
:1012D00002F06CF802494FF000608039086010BDE0
:1012E00088ED00E000380240FFFFF2FE023003000C
:1012F0007CB501210E4802F017F9684602F08EFE17
:1013000001208DF8060000208DF804008DF80500FE
:101310000220084D4FF480548DF807000094694670
:10132000284602F085FE2146284602F00FFE7CBDCD
:10133000010030000004024010B5084C0121204695
:1013400004F0F2FA002807D0FFF72EFD2046BDE892
:101350001040012104F0E5BA10BD0000000001407A
:1013600010B5124802F052F801214FF4880002F043
:10137000DBF80F4C8B220621204604F0C1FA002135
:10138000204604F0C4FA01221146204604F0D3FAA4
:10139000032003F0F5FB00220121192003F0B2FB2A
:1013A0002046BDE81040012104F0B6BAE00000205C
:1013B0000000014070B52A4C1021204604F0DDFCED
:1013C000F8B11021204604F050FCD0B11021204685
:1013D00004F037FC234D284602F022FAC0F1020047
:1013E00082B221492148FFF754FE0021284602F02D
:1013F00061F90221284602F016FA0121284602F07E
:1014000059F940212546204604F0B7FC002825D094
:10141000154916480222891E5030FFF717FE0404B2
:10142000240C14D00F4E0021143E304602F042F935
:10143000022002F007FA2146304602F0F4F90121B9
:10144000284604F0F4FB0121304602F033F9284627
:10145000BDE870400022064904F080BC70BD000069
:10146000001001401C60024062000020280A002099
:1014700006000C0070B52B4C1021204604F07DFCBA
:10148000251500B31021204604F0EFFBD8B1102140
:10149000204604F0D6FB244E304602F0C1F9C0F5D8
:1014A0008060224982B2A1F59060FFF7F2FD002131
:1014B000304602F0FFF82946304602F0B4F9012127
:1014C000304602F0F7F840212646204604F055FC4D
:1014D000002825D016492A46A1F13000FFF7B6FDB5
:1014E0000404240C15D0104D0021143D284602F0B0
:1014F000E1F84FF4003002F0A5F92146284602F049
:1015000092F90121304604F092FB0121284602F0B5
:10151000D1F83046BDE870400022064904F01EBCF8
:1015200070BD0000004800406C600240C80E002002
:10153000C80A002006000C00FEE700000FB47CB5CE
:101540000C0009AD01D0611E00E00021CDE90001D1
:10155000064B6A462946089800F060F9002C02D034
:10156000009A002111707CBC5DF814FB231F000859
:101570000907090E002804DB00F1E02080F80014C0
:10158000704700F00F0000F1E02080F8141D704754
:1015900030B528B1144C031F002021680A4605E02D
:1015A000084630BD9A4203D810465268002AF9D145
:1015B000002800D041680BD00468A3EB0005A542C9
:1015C00004D11B681C440346046002E0436000E051
:1015D00023603AB11C68D51AA54203D115682C4482
:1015E0001C6052685A6030BDD80000200000000026
:1015F00000B583B09FED060B0A4601468DED000B4A
:101600006846FFF73CFA9DED000B03B000BD0000FB
:1016100000000000000000002DE9F04782460F4C5A
:1016200010480D4E0E4F001B4FF0000820F007052C
:101630004FF0010900221146504602F029FF002810
:1016400002D1306810B10020BDE8F0873C60C4E9E9
:101650000058C6F80090EDE7DC000020944500201B
:10166000D80000209047002002E008C8121F08C1DF
:10167000002AFAD170477047002001E001C1121F13
:10168000002AFBD1704700002DE9FF5F82B00021E6
:10169000DDE90430020DDDF840B0034318D044F614
:1016A0001050A2F2FF3242431514119801281FD0A6
:1016B000A5EB0B00401C5FEA000A4FF000064E4FFE
:1016C000DFF83891B046504615D5CAF1000413E052
:1016D000119801244AA3012801D16FEA0B01029855
:1016E000119AC0E90031C0E9024206B0BDE8F09F9E
:1016F000CBF10000DFE704460021404A491842EBE5
:101700000450CDE9001012E0E00707D032463B4616
:1017100040464946FFF76FF88046894632463B46C9
:1017200010461946FFF767F806460F466410002C6E
:10173000EAD1DDE90401DDE90023BAF1000F06DAA0
:10174000FFF759F842464B46FFF755F805E0FFF71B
:1017500026FA42464B46FFF722FA04460E4600227E
:10176000284BFFF7F1F803D84FF0FF30014607E0B0
:101770000022254B20463146FEF796FFFFF78AFAF6
:10178000102409E0002C0ADB0A220023FEF746FDA4
:10179000039B30321A55641E50EA0102F2D1641CD8
:1017A000039AC4F111031444119A012A03D00122AF
:1017B00008430DD10AE0084304D000204FF0110B7C
:1017C000119072E7A3EB0B056D1E0DE05B4504DD88
:1017D0004FF0000205F1010504E003DA4FF00002CA
:1017E000A5F10105002AECD002981199C0E9023157
:1017F000C0E9004579E70000000014400000F03F18
:10180000300000000000F0430000E03F30380A28BC
:1018100001D2012070470020704700002DE9FF4FE2
:1018200095B09A46884606460025EEE1252877D1F0
:1018300000242746F94A0121039400E0044316F8E6
:10184000013F203B01FA03F01042F7D130782A28FB
:1018500011D06FF02F033078A0F13002092A16D88A
:10186000039A44F0020402EB820203EB42021044AA
:10187000761C0390EFE758F8042B0392002A03DA52
:10188000504244F40054039044F00204761C307833
:101890002E2816D116F8010F44F004042A280DD082
:1018A0006FF02F023078A0F13003092B09D807EB35
:1018B000870302EB4303C718761CF3E758F8047B51
:1018C000761C30786C280FD006DC4C2817D068289E
:1018D0000DD06A2814D104E0742810D07A280FD1D2
:1018E0000DE044F400140AE044F4801401E044F4F0
:1018F00040147278824202D104F58014761C761C62
:10190000307866280BD013DC582877D009DC002803
:1019100075D04528F6D04628F4D047281AD193E14F
:1019200018E0632835D0642879D0652812D18BE17E
:10193000702873D008DC6728F1D069286FD06E2832
:101940000DD06F2806D1ACE073282CD0752874D048
:10195000782853D05246179990476D1C54E1C4F330
:101960000250022809D003280DD0D8F8001004280E
:101970000DD00D6008F1040846E1D8F80010EA1710
:10198000C1E90052F6E7D8F800100D80F2E70D70BB
:10199000F0E718F8041B8DF8001000208DF8010006
:1019A000EB46012003E058F804BB4FF0FF3061071D
:1019B0004FF0000102D40DE009F101018946B9425E
:1019C0000FDA8145F8DB1BF809100029F4D108E093
:1019D00009F1010189468142FADB1BF8091000294F
:1019E000F6D103985346A0EB090721463846179ACB
:1019F00000F080FA284400EB090507E044E008E124
:101A00000DE01BF8010B524617999047B9F10109F7
:101A1000F7D2534621463846179AF2E039E00A21B8
:101A2000C4F302524FF0000B0091022A06D058F87E
:101A3000040BC117032A09D00AE023E008F10700CC
:101A400020F00702F2E80201904605E000B2C1175B
:101A5000042A01D140B2C117002906DA0A46002142
:101A6000404261EB02012D2202E0220504D52B2227
:101A70008DF80420012203E0E20701D02022F7E7DD
:101A8000914657E00A2100E010214FF0000B009131
:101A90000BE010214FF0000B44F0040408270091E4
:101AA00003E008204FF0000B0090C4F30252022A1A
:101AB00005D058F8040B0021032A08D008E008F1EB
:101AC000070020F00702F2E80201904603E080B22E
:101AD000042A00D1C0B24FF0000922072AD532787B
:101AE000702A07D0DDF800C08CF0100C5CEA0B0CFB
:101AF00005D00EE040228DF80420012208E050EAD3
:101B0000010306D030238DF804308DF80520022221
:101B10009146009B83F0080353EA0B030AD150EA75
:101B2000010201D1620705D530228DF804204FF063
:101B300001097F1E3278582A04D039A20C920CAACF
:101B400002920BE03BA2F9E75B46009AFEF766FBC8
:101B50000C9B9B5C029A521E0292137050EA010287
:101B6000F2D1029804A9081A00F1200B600702D5EF
:101B700024F4803400E001275F4502DDA7EB0B0071
:101B800000E0002000EB0B01009003984944401A4C
:101B90000390E00306D453462146179A039800F0B9
:101BA000A9F90544002706E001A85246C05D17992F
:101BB00090476D1C7F1C4F45F6DBE0030CD5534668
:101BC0002146179A039800F095F9054404E0302067
:101BD0005246179990476D1C0099481E00900029A5
:101BE000F5DC08E00298029952460078491C0291FF
:101BF000179990476D1CBBF10001ABF1010BF1DCB3
:101C00005BE100F065F90544761C307800287FF42C
:101C10000DAE19B02846BDE8F08F0000092801007C
:101C20003031323334353637383961626364656652
:101C30000000000030313233343536373839414214
:101C40004344454600000000600700D4062708F121
:101C5000070020F00700F0E80223804603F0004C64
:101C60005FEA0C0001D097A009E0200501D596A0FD
:101C700005E0E00701D095A001E0AFF24C00139021
:101C8000307823F0004365280CD006DC452809D0C5
:101C900046281DD047287FD13BE0662818D067280A
:101CA0007AD136E00021112F01DB112000E0781CF1
:101CB000CDE9000104A90CA8FFF7E6FCDDE90D0160
:101CC0000C9A4FF0000B07F10109109200914EE0C1
:101CD0004FF000400097CDE9011004A90CA8FFF7D0
:101CE000D3FCDDE90D020C9B0F994FF0000B9146E0
:101CF0001093009211B9791C00EB0109B7EB0900B0
:101D000003D4C0F1FF3B07F10109A9EB07000190E3
:101D100042E0012F00DA01270021112F01DD1120FF
:101D200000E03846CDE9000104A90CA8FFF7ACFC9F
:101D3000DDE90D010C9A00914FF0000BB9461092AD
:101D400021070FD4009A4A4503DA914601E0A9F130
:101D50000109B9F1010F05DD109AA9F10101515CEA
:101D60003029F4D0B84202DA10F1040F03DA01216D
:101D7000CDE9011010E0002803DC8344A9EB000149
:101D800002E0411C494500DD8946A0EB0B00401CE8
:101D900001904FF000400290200705D4019848457B
:101DA00002DB4FF0FF30019000208DF84B000298CD
:101DB0000DF14B07B0F1004F25D002200C902B20E5
:101DC0000D90029800280CDA404202902D200D90D0
:101DD00007E00A210298FEF7CFFD3031029007F8A4
:101DE000011D0C99481E0C900029F2DC0298002875
:101DF000EFD1791E0D980870307800F0200040F087
:101E0000450007F8020D11A8C01BC01D02901398D1
:101E1000007800B1012000EB0901019801EBE071AD
:101E2000029801440398401A401E0390E00306D430
:101E300053462146179A039800F05CF8054413981E
:101E4000007818B15246179990476D1CE00323D5CE
:101E500053462146179A039800F04CF805441BE0BE
:101E6000BBF1000F07DB0098584504DD1098179967
:101E700010F80B0001E01799302052469047019866
:101E80000BF1010B401E05F10105019004D12E203C
:101E90005246179990476D1CB9F10001A9F101094B
:101EA000DEDC05E017F8010B5246179990476D1CD0
:101EB0000299481E02900029F4DC53462146179AE5
:101EC00003989EE62D0000002B000000200000007B
:101ED0002DE9F041044600251E461746880404D427
:101EE00005E039462020B0476D1C641EF9D5284610
:101EF000BDE8F0812DE9F041044600251E469046DC
:101F0000C80301D5302700E02027880404D505E068
:101F100041463846B0476D1C641EF9D52846BDE8D9
:101F2000F0814A68002A06D00A68531C0B601070C2
:101F30004868401E486070470B78426863F3082287
:101F400042604B78826863F3410282608B788268DA
:101F500063F3CB228260C978C26A491E61F31852CA
:101F6000C2620921C0F8D010704700210170417091
:101F700081700121C1707047816841F00801816062
:101F800070478068000701D5012070470020704726
:101F9000816841F00401816070478068400701D585
:101FA000012070470020704707490378D1F80423C7
:101FB00063F31342C1F804234278D1F8040362F3B7
:101FC000D750C1F804037047002001400021017080
:101FD000417070471CB5002001F0BEF901A8FFF761
:101FE000F5FF00248DF804408DF8054001A8FFF7A7
:101FF000DBFF6846FFF7B9FF01208DF800008DF880
:1020000001008DF8024002201F4C8DF80300694644
:102010002046FFF791FF0021204600F00CF9022333
:1020200001220821204600F08DF802231A460921DA
:10203000204600F087F800220721204600F0EDF846
:102040000121204600F056F80121204600F057F803
:102050000121204600F058F84021204600F059F8B0
:102060000028F9D02046FFF787FF2046FFF789FFB9
:102070000028FAD12046FFF78BFF2046FFF78DFF9F
:102080000028FAD11CBD00000020014070B5164C9C
:1020900000256068012811D114499022A1F507702C
:1020A0006560FEF7F2F8124800F55471C1F80600B9
:1020B000032002F00DFD2069401C206101F040FF6B
:1020C000D4E90623801A61EB03014FF47A72801A77
:1020D00071F1000006D301F033FFC4E90601206965
:1020E000C4E9045070BD000008000020C8080020AA
:1020F000AC060020826861F3082282607047826823
:1021000061F3492282607047826861F30002826055
:1021100070470246002012680A4200D00120704732
:1021200010B503F095F901F015FF01F0C9FAFFF7BA
:1021300051FFBDE810400121014800F077B80000D0
:102140000020014070B507240A2908D2056901EB77
:102150004106B440A543B3402B43036116E0142964
:102160000AD2C568A1F10A0606EB4606B440A543AB
:10217000B3402B43C36009E0056DA1F1140606EBE3
:102180004606B440A543B3402B4303651F23072AEB
:1021900009D2446B521E02EB820293409C43914051
:1021A0002143416370BD0D2A09D2046BD21F02EB9B
:1021B000820293409C4391402143016370BD112AE8
:1021C00009D2C46A0D3A02EB820293409C439140CB
:1021D0002143C16270BD172A09D2446D113A02EB46
:1021E000820293409C4391402143416570BD1D2A6A
:1021F00009D2846D173A02EB820293409C439140CE
:102200002143816570BDC46D1D3A02EB820293408B
:102210009C4391402143C16570BD836861F31B639A
:102220008360816862F31D7181607047826861F329
:102230009E7282607047426861F319624260704723
:1022400000B585B0684601F0C9FC002806D0BDF88D
:102250000000A0F525415A3902D0002005B000BD8C
:102260000120FBE710B508B101F058FCBDE81040B3
:1022700000F010B80248002181600170C170704701
:10228000B80000200248012141700021C170704750
:10229000B800002070B58CB0FFF7D2FF00B101206C
:1022A000244C20700126E67020780025C0B10AA8D1
:1022B000009009AB08AA07A906A800F039FA10B9DE
:1022C00000F0F4F9257000F0ADFBA06010B180893A
:1022D000022800D2257000F093F920B9257002E0A1
:1022E00000F0E4F9A5601348401D00F04BF801A888
:1022F00000F00CFA2178104819B1BDF806100170F1
:1023000000E0067006700D4CFF25ADF80E50BDF8CC
:102310000A002080BDF808106180BDF80C20A28062
:102320004FF48053E3802581009502F001FA0CB050
:1023300070BD0000B8000020B000002070450020F3
:1023400010B5040002D04AF25A5000E000200749BC
:102350000880084601F05AFC002806D00CB1012084
:1023600000E0002002490870012010BDDA40002082
:10237000B8000020002803D04178007800F03EBD6E
:102380007047000010B5040003D001F04BFB10B102
:1023900009E0002010BD204600F01EF8204601F0A4
:1023A0005BFB0028F6D004482188A0F80510401DEA
:1023B000FFF7E0FF012010BDB800002010B500F0CD
:1023C00013F8002805D0034801F046FB002800D090
:1023D000012010BDBD000020002803D002210170A3
:1023E0000A2141707047000010B5002808D0054947
:1023F00002780A70407848700846FFF7BBFF01205A
:1024000010BD0000BD00002010B504000BD001F08D
:1024100041FB50B1204600F044F8204600F00CF893
:1024200018B1012010BD002010BD204600F048F872
:10243000204600F0A3F8F4E710B504002FD023786D
:102440006BB394F8212052B394F8321039B394F856
:102450003A0020B3FF2B22D0FF2A20D0FF291ED024
:10246000FF281CD0212200212046FDF747FFB0B1F4
:102470001122002104F12100FDF740FF78B108226C
:10248000002104F13200FDF739FF40B10F22002195
:1024900004F13A00FDF732FF08B1012010BD002021
:1024A00010BD00280AD0002100F8201F4174417699
:1024B00080F8281080F8321080F83C107047000037
:1024C00010B586B004004FF0000001900290039018
:1024D00004902FD05D212046FDF7F0FE16A01022BB
:1024E000006820603920207115A104F12100FDF75A
:1024F000CCFE18A00D220168C4F832108088E08656
:1025000016A104F13A00FDF7C0FE0C20034600902E
:1025100016A2102101A8FFF711F801A8FDF7D9FEB6
:10252000024601A904F14900FDF7AFFE11A00068C1
:10253000C4F8530006B010BD4A4A303039000000DC
:10254000464130303630473141373130303030312C
:102550000000000056312E302E31000056312E3052
:102560005F323032353036323700000025752C2589
:102570007500000056312E300000000000B599B003
:10258000002812D001465D226846FDF77EFE6846AF
:10259000FFF787FF6846FFF74FFF002805D0684622
:1025A00001F08CFA002800D0012019B000BD000015
:1025B00000487047C4000020002802D0014900688C
:1025C000C8607047B800002010B54FF45871074834
:1025D000FDF774FE01F0B6FA002805D00020FFF7E1
:1025E000AFFE002800D0012010BD0000EE4000200A
:1025F00000487047EE4000204FF4587070470000CC
:1026000010B54FF4D871064801F0A8FA08B10120BE
:1026100010BD4FF458710248FDF750FE002010BD68
:10262000EE40002010B500F019F8002813D04FF448
:10263000D8742146084801F0ADFA00280BD0214695
:10264000054801F08BFA002805D00120FFF778FE3D
:10265000002800D0012010BDEE40002010B518B1B8
:102660004FF45872914201D0002010BD014602483B
:10267000FDF70BFE012010BDEE40002008B500283C
:1026800011D00949C2884FF480530A8082884A8059
:1026900002898A80CB8042890A81009202898188DE
:1026A000C08802F045F808BD7045002010B586B01E
:1026B00014216846FDF702FE4FF47A70ADF804006D
:1026C00042F21070ADF8060040F21450ADF8080068
:1026D000FF20ADF80A000024ADF800406846FFF77F
:1026E000CDFF09480480BDF804108180BDF80610B4
:1026F000C180BDF808100181BDF80A10418101F0C8
:1027000085FA06B010BD0000DA40002000280BD08A
:102710000649CA88C2808A8882800A8902814A89D9
:10272000428149884180012070470000DA40002042
:102730002DE9F04186B01C46DDF8308015460E4686
:10274000070016D0AEB1A5B19CB15FEA080010D069
:10275000684601F043FA00280CD0BDF80000A0F54F
:1027600025415A3905D1BDF80400BDF8061088424C
:1027700003D3002006B0BDE8F0813880BDF8060024
:102780003080BDF808002880BDF80A002080BDF820
:102790000210A8F800106846FFF770FF0120E9E773
:1027A00070B586B00D46040025D025B3684601F00B
:1027B00015FA082608B3BDF806002070BDF806001B
:1027C000000A6070BDF80400A070BDF80400000AA3
:1027D000E070BDF808002071BDF80800000A6071C3
:1027E000BDF80A00A071BDF80A00000AE0712E8051
:1027F000012006B070BD0020FBE7FF220821204623
:10280000FDF755FD2E80F6E7C8B1C1B10D4A9379A9
:102810000370D3881B0A43701379837093881B0A53
:10282000C370137A037113891B0A4371937A8371FE
:102830005289120AC27108200880012070470020C6
:1028400070470000DA40002000B585B000F034F891
:10285000002813D0684601F0C1F9094908B1BDF854
:1028600000000880064801F0D1F9002806D068462B
:1028700001F0B4F96846FFF701FF012005B000BD83
:10288000DA40002010B5002813D00A4982888A80D7
:10289000C288CA8002890A8142894A814088488068
:1028A0000846FFF7EBFE034801F0B0F9002800D01E
:1028B000012010BDDA40002010B580B108290ED3E8
:1028C000028841888388C488914208D20548818063
:1028D000C28003814481FFF7D1FE012010BD00209A
:1028E00010BD0000DA40002010B504461348144A19
:1028F00001214460204601F0B3FF124A0221204624
:1029000001F0AEFF104AAA21204601F0A9FF0F4AAC
:10291000FB21204601F0A4FF0D49204601F0FEFFF7
:102920000023F02221460B4802F08FF8BDE810404A
:10293000094B0A4A0A49074802F0B6B8B00000201D
:10294000FD42000895420008C94200083D430008C6
:102950009D29000818340020955900084D59000899
:10296000D95900081FB54FF480620A4BCDE90032F7
:102970000021A3F58063CDE90201A3F58061A1F1F7
:10298000840001F04DFF04B00348BDE81040FFF79C
:10299000ABBF0000D03C00204C3400207CB5084682
:1029A000072A27D30168009101798DF804109DF85A
:1029B000021002291ED1BDF80310441D4A1F95B212
:1029C00042181288ADF8002001F004FFBDF8001095
:1029D000884211D074B1032D0CD320783D2801D04A
:1029E0003F2807D160787B2804D1601910F8010CCA
:1029F0007D2801D000207CBD2946204601F074FBD3
:102A000001207CBD064910B5002088810A39886103
:102A10008883034801F02FF9002800D0012010BD61
:102A2000DA40002010B50D4801F014F908B10B4848
:102A300010BD0A4800214FF47A720180828042F270
:102A40001072C28040F214520281FF2242818181C1
:102A50000A3881618183084610BD0000DA400020F9
:102A600030B585B00D4604001CD0DDB1684601F0DC
:102A7000F1F8C8B1BDF80C002070BDF80C000DF1E4
:102A80000E01000A6070BDF80C004200A01CFDF7AA
:102A9000FCFBBDF80C00022101EB40002880012066
:102AA00005B030BD0020FBE700202880FAE70000D9
:102AB00070B50D46A8B1A5B10B4C217B00F8011BE8
:102AC000A189090A00F8011BA1894A0004F10E013D
:102AD000FDF7DBFBA089022101EB400028800120EB
:102AE00070BD002070BD0000DA40002010B500F07D
:102AF0000BF8002805D0034801F0BDF8002800D0ED
:102B0000012010BDDA40002010B520B1022902D307
:102B10000178032901D9002010BD074A00239181C3
:102B20000A3A936193834A00411C03480E30FDF733
:102B3000ACFB012010BD0000DA4000201FB50E489C
:102B40000121817041719021A0F8031014380C21EB
:102B500001704170A0F6F80181609031C160903140
:102B600001610648FFF7FEFE054B0FCB8DE80F0015
:102B70006846FFF777FB1FBDFC090020B54A000837
:102B8000C85F0008002205E0835CFF2B01D0002015
:102B90007047521C8A42F7D3012070471CB5044687
:102BA0001848012150F8240000F0BEFC684601F0EE
:102BB00035FA01208DF8070000218DF804108DF8FA
:102BC00006001048143830F8140000900D488DF8B5
:102BD00005100C38694650F8240001F029FA0A4C17
:102BE0008021204601F0B4F98021204601F0AEF9A1
:102BF0008021204601F0ACF98021204601F0A6F9A1
:102C00001CBD0000540000200004024010B530B18B
:102C1000036823B1D0E90121914201D204E00020F0
:102C200010BD491C816020B1914202D25C5C202C15
:102C3000F7D99142F4D1491E816010BD2DE9F041D0
:102C400004460027104E1BE0A0892568C0050BD460
:102C5000A06820B1FFF7F2FFA089C00504D4206965
:102C600010B1716888472761A089800504D4206A63
:102C700010B17168884727627168204688472C46E2
:102C8000002CE1D1BDE8F08188000020002901DAA4
:102C90000020704701F00CB901004FF0000001D096
:102CA000896803E0002070470968401C0029FBD1B7
:102CB0007047002201F007B9002803D0007B2028CC
:102CC00001D00020704701207047002803D0007B0E
:102CD000102801D0002070470120704710B501680E
:102CE00028208847040002D02821FDF7E7FA204673
:102CF00010BD0022114600F06FB800002DE9F0472A
:102D000088B00F4604469A4616461C216846FDF7D1
:102D1000D5FA2F480025002C0560456055D0814626
:102D2000E7B3CDE900470295D9E90212D9F81000BE
:102D30000491CDE9052009F10800FFF7CFFF5FEA14
:102D400000082BD000986F4608B1029808B1002700
:102D50000BE00198042808D903221EA10098FDF772
:102D6000E4FA10B90298C01C02903846FFF74EFFF3
:102D70000146404602F00CFA68B1BAF1000F13D0D8
:102D80006846FFF743FFDDE90101814203D2029962
:102D90000098405C40B14046FFF750FFDDE901106C
:102DA00088420AD205460BE01EB1029900980844F9
:102DB0003060404608B0BDE8F087081E00D0451ED0
:102DC0000EB160193060C9E900450020F2E700004B
:102DD00080000020EFBBBF0070B515460E46040012
:102DE00009D0FDF776FA411C2B4632462046BDE855
:102DF0007040FFF783BF002070BD0000014A1070D3
:102E0000517070479800002070B588B001212248A9
:102E100000F08AFB04A800F007F900248DF81440A4
:102E20001E4E8DF81540012504948DF8165004A906
:102E3000304600F069F81E20ADF818008DF81A40F1
:102E400005208DF81B008DF81C4006A9304600F0C7
:102E5000ADF88DF800508DF803408DF802408DF8E4
:102E60000440ADF808408DF80140ADF80640ADF8DB
:102E70000A40ADF80C406946304600F0DEF800220A
:102E80000221142001F03EFE01220221304600F012
:102E9000E3F908B070BD0000190040000064004074
:102EA0001CB501214FF4401000F03EFB684601F0D4
:102EB000B5F801208DF8070000208DF804000221EC
:102EC0008DF806104FF4C0510E4C00918DF805009E
:102ED0006946204601F0ACF809220C21204601F099
:102EE000D9F809220B21204601F0D4F8FEF700FAA8
:102EF000642000F0B9FBFFF787FFBDE81C40C82045
:102F000000F0B2BB0000024010B50368002223F0BD
:102F100002030360036843F0010303604FF6FF738D
:102F200000E0521C4468E40701D19A42F9D142689A
:102F3000D20737D04C78026864F3C71202608C78ED
:102F4000026864F386120260CC78026864F345126A
:102F500002600C79026864F3041202604C79026822
:102F600064F3C30202608C79026864F38202026037
:102F70000A78C46962F39E74C46109784A08C16919
:102F800062F3DF71C161016821F00101016000217C
:102F900000E0491C4268D20701D09942F9D140684B
:102FA000C00701D0002010BD012010BD10B503687E
:102FB000002223F002030360036843F0010303606F
:102FC0004FF6FF7300E0521C4468E40701D19A42B7
:102FD000F9D14268D20723D00A88C469521E62F32D
:102FE0000B04C4618C78C26964F31962C261CC7845
:102FF000C26964F31342C2610A79C16962F316516E
:10300000C161016821F001010160002100E0491C5B
:103010004268D20701D09942F9D14068C00701D077
:10302000002010BD012010BD002141708170C170D1
:103030000171417181710170704730B5CB78012207
:103040009A40D0F8003243F00103C0F80032D0F8C3
:103050001C329343C0F81C320B7913B1012B48D1B9
:1030600022E0D0F80C329343C0F80C32CC788B8934
:1030700000EBC4041B04C4F84032CB7800EBC3035C
:10308000D3F840420D892C43C3F84042CC784B8999
:1030900000EBC4041B04C4F84432CB7800EBC30338
:1030A000D3F84442CD8821E0D0F80C321343C0F865
:1030B0000C32CC78CB8800EBC4041B04C4F840323B
:1030C000CB7800EBC303D3F840420D892C43C3F8FF
:1030D0004042CC784B8900EBC4041B04C4F8443252
:1030E000CB7800EBC303D3F844428D892C43C3F85B
:1030F00044424B7813B1012B09D103E0D0F80432DC
:10310000934302E0D0F804321343C0F804328B78C2
:1031100013B1012B09D103E0D0F81432934302E03C
:10312000D0F814321343C0F81432097829B10129B8
:1031300008D1D0F81C12114302E0D0F81C129143C0
:10314000C0F81C12D0F8001221F00101C0F80012E2
:1031500030BD000030B510220823042412290BD200
:10316000DFE801F00A0909090B090F11140A171900
:103170000A1B1D1F2123446030BD44600021816172
:1031800030BD012112E04FF480710FE04FF4803127
:103190000CE0C36030BDC26030BD036130BD026170
:1031A00030BD436030BD426030BD0149816030BDFB
:1031B00001010100002212294CD2DFE801F04B0985
:1031C0000B0F11161A1E2226282A2C3034383A40AA
:1031D00080690FE08069C0F340023BE0806905E050
:1031E000806910F0700F34D134E04068C0F3800281
:1031F00030E0806800F001022CE08068C0F300221B
:1032000028E08068C0F3004224E0C06804E0C068A1
:1032100006E0C06808E0006980071AD11AE000697A
:10322000C0F3C00216E00069C0F3001212E040686B
:10323000F6E7416889070CD44068C00607E081685A
:10324000490106D48168090103D48068C0000028C0
:1032500000DA012210467047002A426901D00A4371
:1032600000E08A434261704710B400EB0113D3F8C9
:10327000B041C4F3800414729CB31CB1D3F8B041C4
:10328000E4085460D3F8B041C4F340045472D3F856
:10329000B44104F00F049472D3F8B441240AD474F6
:1032A000D3F8B841D472D3F8B841240A1473D3F8D0
:1032B000B841240C5473D3F8B841240E9473D3F856
:1032C000BC41D473D3F8BC41240A1474D3F8BC4174
:1032D000240C5474D3F8BC311B0E937410BC00F052
:1032E00005B8D3F8B041640D1460CBE7202219B1C2
:1032F000012900D102617047C260704770B500219A
:10330000041E28D0A52020705A2060709078A070EC
:10331000D078801DE070B2F80300801D000A207193
:1033200050796071062507E0D2F80600405C6055D0
:103330006D1C491CADB289B2B2F803008842F3D8C3
:1033400029462046FDF738FE60556D1CA9B2000ADB
:103350006054491C88B270BD02490A6860F3CF32DC
:103360000A607047A038024000B50246012000F014
:103370001DF80548016862F30711016000205DF83F
:1033800004EB00F013B800000838024002490A6854
:1033900060F38C220A6070470838024002490A68CC
:1033A00060F34F320A60704708380240054901282F
:1033B000086803D020F030000860704740F030000B
:1033C000FAE70000A43802400F4A052810D2DFE8CF
:1033D00000F003070B101300106861F3000006E013
:1033E000106861F3104002E0106861F3186010602B
:1033F00070470548703001E003487430026861F39B
:1034000000020260704700000038024070B50446B8
:1034100000F00AF901002C482C4A04D0012913D0ED
:1034200002292FD116E02949091F0B685B0403D537
:103430000968C90400D52648206010682168C0F3D7
:103440000240C14021601EE020601168C1F3C2410A
:10345000C84017E01D49A0390A680A68C2F38813FA
:103460000A68096802F00F021A4EC1F30241715C4A
:1034700012FB01F2A0FB03010023FCF7CFFE490879
:103480004FEA3000206014490868124AC0F3031064
:1034900002F11602125C206820FA02F060600A68ED
:1034A0000C4BC2F3822203F106039A5C20FA02F26B
:1034B000E260096803F10802C1F34231515C20FA6D
:1034C00001F0A06070BD000000127A00A438024034
:1034D000006CDC02EE5F0008083802400146002064
:1034E00001F01F0301229A40044B03EB1141D1F874
:1034F00000188A4300D101207047000000300240CC
:1035000030B500244FF4405500E0641C1120FFF753
:10351000E5FF012801D0AC42F7D31120FFF7DEFF11
:10352000012800D0002030BD10B5094C00F01F0369
:1035300001229A4004EB10400129D0F8001804D071
:1035400031EA0201C0F8001810BD1143FAE700008B
:103550000030024030B520B90B4C256845F4805549
:103560002560094C9C3C256860F3965525602068D1
:1035700061F38E102060206862F3030020602068F1
:1035800063F31240206030BDA038024000B5012036
:10359000FFF70CFF1848016841F001010160016864
:1035A0008907FCD5144908310A6822F003020A6031
:1035B0000A6812F00C0FFBD10268104B1A4002602F
:1035C0004FF0804008600C490D48091D08600A480A
:1035D000A030016801F4A0410160016841F470214C
:1035E000016005494FF41F000C31086000205DF8B0
:1035F00004EBFFF7DBBE000000380240FFFFF2FEE5
:103600000230030000B502460120FFF7CFFE054857
:10361000016862F30101016000205DF804EBFFF72F
:10362000C5BE00000838024002480068C0F38100AF
:10363000704700000838024002000A494FF00000BD
:1036400007D0012A09D0022A02D10868C0F301106C
:103650007047086800F0030070470868C0F38100F5
:1036600070470000683802404FF4FA71484300F098
:1036700001B8000030B50D4A0D4B4FF0E024126840
:103680000021B2FBF3F3A2694343A0699042FCD04E
:1036900002D2A2EB000203E06569A5EB00052A4413
:1036A000114402469942F0D330BD0000340000209E
:1036B00040420F00026861F30002026070470000A0
:1036C00010B5002286B011460B2001F01BFA194CF0
:1036D000204600F0F9F8684600F0A7F801218DF8BF
:1036E0000F1000228DF80D108DF80E10ADF8082087
:1036F0008DF80C2010480222019010488DF81120FE
:1037000000908DF81010ADF80A206946204600F0B0
:10371000A9F808480121303800F004F905480521CE
:10372000DC3000F006F901212046FFF7C3FF06B0A8
:1037300010BD000030600240780000204C200140A5
:103740002DE9F04F0D46064685B001213048FFF7C0
:10375000EBFE01212F4800F0E5F82E48083000F07C
:10376000B3F8684600F061F800248DF80F40012797
:10377000DFF8A4908DF80D704FF00208CDE90096A7
:103780002448ADF80A508DF80E408DF811804FF0A6
:10379000100A8DF80C408DF81040ADF808A069466D
:1037A000083000F05FF8DFF874B00B21584600F0E5
:1037B000C0F8184801210830FFF77CFF1548083091
:1037C00000F082F8684600F030F88DF80F408DF870
:1037D0000D70CDE900960F48ADF80A508DF80E40F7
:1037E0008DF811808DF80C408DF81040ADF808A0D0
:1037F0006946083000F036F80B21584600F099F879
:10380000044801210830FFF755FF05B0BDE8F08FEF
:1038100018003000006402400C3001400465024092
:10382000406880B27047416070470021016041608C
:1038300001814181017341738173C17301744174CA
:1038400070470000B0F1805F04D9044920F0704057
:1038500008607047024948607047000004640240F5
:103860000060024002684BF6EF731A400260026883
:103870000B891A4302604B7C026863F30D320260CD
:10388000CB7B026863F38B2202608B7B026863F35D
:10389000092202604B7B026863F3C71202600B7B54
:1038A000026863F3861202600B7C026863F34512C0
:1038B00002604B89426863F30F0242600A688260CB
:1038C0004968C16070470000016821F00101016092
:1038D0000021016041608160C16040F2FF6100EA47
:1038E0000102C0B214230F210838B2F5C16F08D20B
:1038F000B0FBF3F08000814008484268114341600A
:103900007047B2F5D16FFBD2B0FBF3F0800081407D
:1039100003480268114301607047000000600240E4
:1039200004640240D0F8002161F30002C0F80021D5
:103930007047026861F306020260704710B50446E2
:1039400000F020FA4FF0804000F04EF8042804D038
:10395000012805D0022803D005E000F029F80AE08C
:10396000142000F00DF8204600F0F6F9044600F0AF
:103970001FF8032C01D0012010BD002010BD000055
:1039800001490860704700000C3C024010B5074C2C
:10399000226842F00102226001804FF4801000F0A2
:1039A00023F8216821F00101216010BD103C024084
:1039B0000248016841F0800101607047103C0240FC
:1039C000084903200A68D20701D0002070470A681E
:1039D000520701D5012070470968C906FBD50220AE
:1039E000704700000C3C024000B50346FFF7E8FFBB
:1039F00003E000BFFFF7E4FF5B1E18B1002B00D10E
:103A0000042000BD002BF5D1FAE70000082900D200
:103A100001B90821024AD26802B11047002070475C
:103A20007C4500201CB5040011D0082269460948D5
:103A300000F048FB002809D00098411C02D10199F0
:103A4000491C04D020700198607001201CBD00202A
:103A50001CBD000000E800081CB5002817D0017844
:103A6000009140780A4C01904FF40061204600F02C
:103A700043F800280BD008226946204600F02CFBB2
:103A8000002804D008226946204600F031F91CBD08
:103A900000E8000870B5040005D0074D5D212846F8
:103AA000FFF7B4FF08B1002070BD21462846BDE8ED
:103AB00070405D2200F006BB00F0000870B5040005
:103AC00015D00C4D4FF40061284600F015F8002881
:103AD0000ED05D222146284600F0FEFA002807D0CD
:103AE00021462846BDE870405D2200F001B9002063
:103AF00070BD000000F0000870B5074A0C4605468E
:103B000092683AB1904728B121462846BDE87040F6
:103B1000FFF77CBF002070BD7C45002010B5002859
:103B200003D01DC8014981E81D0010BD7C4500205F
:103B3000002804D001461422014800F0C3BA70479F
:103B400000F8000810B54FF458710348FFF7D4FF90
:103B5000002800D0012010BD0000010870B505004C
:103B60004FEA41040BD0B1F5D87F08D1B4F5587FA6
:103B700005D8074E21463046FFF748FF08B1002020
:103B800070BD224629463046BDE8704000F09ABA22
:103B90000000010870B505004FEA410406D0B1F5F8
:103BA000D87F03D14FF458718C4201D9002070BDE9
:103BB000094E3046FFF7A0FF0028F8D022462946DC
:103BC000304600F089FA0028F1D0224629463046D6
:103BD000BDE8704000F08CB80000010810B5044644
:103BE000FFF7A6FF00280ED0A1884FF6FF70814294
:103BF0000AD1E188814207D12189814204D16189BA
:103C0000814201D1002010BD012010BD10B586B049
:103C1000044614216846FCF751FBCCB16846FFF717
:103C200087FF2088ADF80000A088ADF80400E08888
:103C3000ADF806002089ADF808006089ADF80A00EB
:103C40006088ADF80200684600F034F806B010BD98
:103C50000020FBE710B50446FFF76AFF002807D0F5
:103C6000A089A0F57F41FF3901D0032801D90020A8
:103C700010BD012010BD10B586B004461421684661
:103C8000FCF71CFB14B1A089032802D9002006B060
:103C900010BD6846FFF74CFFA089ADF80C00D4F8C2
:103CA0000E00CDF80E00608AADF81200684600F0F4
:103CB00001F8ECE770B5040015D00C4D4FF400612D
:103CC0002846FFF719FF00280ED014222146284667
:103CD00000F002FA002807D021462846BDE87040CF
:103CE000142200F005B8002070BD000000F80008A4
:103CF0002DE9F04190B0164680460F004FF00004C9
:103D000018D192B918E0351B402D00D3402508EB9F
:103D100004002A46694600F0D5F9002806D0391972
:103D20002A466846FCF7F4FA18B1002010B0BDE846
:103D3000F0812C44B442E6D30120F7E710B500230C
:103D400005E000BF30F8024B21F813405B1C9342A2
:103D5000F8D3002010BD000010B5094C216841F0D7
:103D600002012160211D0860206840F040002060B1
:103D70000807FFF739FE216821F00201216010BD1C
:103D8000103C02400348024901600349016070474A
:103D900023016745043C0240AB89EFCD2DE9F74F85
:103DA00015468846FFF7EEFF0098A0F10060C0F3CB
:103DB0004906C70AC6F58064A54200D82C46DFF83C
:103DC000BCA04FF4806B00BF4FF0006000EBC72039
:103DD00081465A462949FFF7B1FF00204FF6FF718F
:103DE00005E033183AF813208A4202D1401CA04261
:103DF000F7D3A0422AD24FF08040FFF7F5FD01280B
:103E000009D0022807D004281BD04846FFF7A4FF9A
:103E1000032816D103E01420FFF7B2FDF5E70020D8
:103E2000514605E038F810208319401C21F8132072
:103E3000A042F7D3114948465A4600BF00F020F887
:103E400040B1FFF7B5FD0120BDE8FE8F2246414697
:103E50000098F3E7A5420DD0009808EB440800EB6A
:103E600044002D1B00265C467F1C0090A542ABD869
:103E70002C46A9E7FFF79CFD0020E5E7F022002093
:103E80002DE9F041174606460D4600240CE000BF20
:103E900035F814103046FFF779FD032802D00120D1
:103EA000BDE8F081641CB61CBC42F1D30020F7E7EA
:103EB000002807D0806801E00068491E002801D072
:103EC0000029F9D170472DE9F0418846A8B3B8F12F
:103ED000000F33D084680AB90AE024686CB3216A01
:103EE00059B34046FCF7FCF90028F6D120E02468DD
:103EF0001CB3266A5FEA0805F9D0002EF7D0B54258
:103F000018D002E098B16D1C761C2878FCF7B7F940
:103F100007463078FCF7B3F987422878F2D0FCF7EF
:103F2000AEF905463078FCF7AAF98542DFD124B115
:103F3000206A10B12046BDE8F081FFE70020FAE7D3
:103F4000014908684968704738000020816270475D
:103F5000816170477CB5684600F060F80120094D2A
:103F6000032400908DF806406946284600F060F86A
:103F7000022000908DF806406946284600F058F867
:103F80007CBD0000000402407CB501214FF44010CC
:103F9000FFF7CAFA684600F041F800208DF80400E7
:103FA00001248DF80740022510201B4E8DF8065085
:103FB00000908DF805506946304600F039F805222A
:103FC0000421304600F066F8202000908DF805505E
:103FD0006946304600F02CF805221146304600F0C4
:103FE00059F8402000908DF805406946304600F0B1
:103FF0001FF805220621304600F04CF88020009082
:104000008DF805406946304600F012F80522072178
:10401000304600F03FF87CBD000002404FF6FF71D3
:10402000016000218171017141710121C1717047ED
:10403000F0B50B8800229BB229E0DC0724D006688B
:1040400055000324AC40A64306608E790768AE4055
:104050003E430660466801279740BE434660466877
:104060000F7997403E4346608668A6438660CE79C6
:104070008768AE403E438660C668A643C6604C79FA
:10408000AC40C5682C43C4605B08521C92B2002B44
:10409000D3D1F0BD4B0710B5DB0E9A40CC084FF0E2
:1040A0000F0101FA03F106D0436A8B434362416A70
:1040B0001143416210BD036A8B430362016A1143DD
:1040C000016210BD034B1B680BB15208184700205A
:1040D000704700007C450020024B5B6803B1184725
:1040E000002070477C450020F0B58BB04FF0FF34C6
:1040F00000B302291ED301783D297DD1401CFEF773
:10410000F8FD060016D0FEF753FA006808904AA1A1
:104110003046FEF7CEFD10B1007D8DF8200048A19D
:104120003046FEF7C6FD70B19DF8211040690129A7
:1041300003D006E020460BB0F0BD10B901218DF888
:1041400022108DF8210040A13046FEF7B2FD10B1DB
:10415000007D8DF823003EA13046FEF7AAFD0746FC
:104160003DA13046FEF7A5FD054667B33846FEF78C
:10417000A3FD40B33846FEF78FFD044603A8FEF7C3
:10418000C5FA00B3012C06DB00213846FEF77EFDA0
:10419000808AADF81200022C06DB01213846FEF7BA
:1041A00075FD808AADF8100055B1686940B1052CE5
:1041B00006DB04213846FEF769FD808AADF816005B
:1041C00003A8FEF75FFB27A13046FEF772FD044609
:1041D00028A13046FEF76DFD054654EA05000FD0D4
:1041E00003A8FEF7CFF814B1207D8DF80C0015B1AF
:1041F000287D8DF80D0000E01CE003A8FEF7F4F820
:104200001FA13046FEF755FD04000DD0FEF75DFD01
:1042100050B11DA12069FCF763F828B96846FEF784
:10422000B1F86846FEF7CAF808A8FEF7C5F93046A7
:10423000FEF704FD00207EE76C65645F7377000085
:1042400074785F73770000007069636B5F73770049
:104250006D617468000000006D6174685F66756C64
:104260006C00000063726565705F737472656E67E1
:104270007468000063726565705F6C6576656C00DC
:10428000666C61736800000063726565705F7772C9
:1042900069746500F0B41046032B11D3C11CDB1EFA
:1042A0009AB2084C0578002314F83360AE4204D16A
:1042B00004EBC3035B68F0BC18475B1C032BF3D310
:1042C000F0BC704714600008F0B41046032B11D303
:1042D000C11CDB1E9AB2084C0578002314F8336029
:1042E000AE4204D104EBC3035B68F0BC18475B1C0F
:1042F000022BF3D3F0BC70472C60000830B585B0BA
:104300001446032B16D30C4D2078297888420ED002
:1043100028706846FEF7FAF948B140F6FF70ADF82C
:104320000A002878ADF802006846FEF7ABFAB4F848
:104330000100688005B030BDB000002011461A466B
:10434000014800F0FCBA0000183400202DE9F047C5
:10435000174D06464FF480412846FFF7F7FDDFF87A
:104360005490AF1539464846FFF7F0FD4FF4004A28
:1043700051462846FFF7EAFDB84600244F4609E0BB
:1043800041463846FFF7E4FD41463846FFF7DEFD7B
:10439000641CE4B2B442F3D3544651462846FFF7B6
:1043A000D7FD21462846BDE8F047FFF7CFBD000006
:1043B00000040240000002401CB501214FF44010EF
:1043C000FFF7B2F801211048FFF7AEF86846FFF793
:1043D00025FE01208DF8070000218DF804108DF8CE
:1043E0000600000200908DF8051069460748FFF7A7
:1043F0001FFE4FF46040009069460548FFF718FE25
:104400002020FFF7A3FF1CBD010030000000024088
:10441000000402402DE9F047DFF86C9007464FF4A6
:10442000804841464846FFF793FD184E4FF480758B
:1044300029463046FFF78CFD0020401EFDD229465C
:104440003046FFF783FDC2460024C8460DE05146C2
:104450004046FFF77BFD29463046FFF779FD2946A8
:104460003046FFF773FD641CE4B2BC42EFD34FF457
:104470000045294644464046FFF76AFD2946204646
:10448000BDE8F047FFF762BD0004024000000240B3
:104490002DE9F0410B3020F00706104D19E020689F
:1044A000B04215D3B0420AD9871B201DD4F804802E
:1044B000FBF7EBFEA019C0E90078286004E0606813
:1044C0002860201DFBF7E1FE201D2660BDE8F0817D
:1044D000251D2C68002CE2D10020F7E7D800002031
:1044E00010B5034800F0CEFF012800D0002010BD19
:1044F000080A002001F04EF9032000F041FB01F012
:10450000DFF90020FEF74AFBFEF7CAFCFDF708FEC4
:10451000FCF75CFE01F006F8FFF74EFF00F0ECFA46
:10452000FFF7DEFF0A490860FEF708FB094801F0C3
:1045300061FB4FF47A70FFF797F8FCF711FF012049
:10454000FFF792F801F010F8FDF7A0FDF7E7000083
:104550000000002080841E002DE9F0410446DDF8B3
:1045600018C0002000250026BCF1000F03D0BCF1CC
:10457000010F65D134E00D462FE063B1012B28D146
:1045800034F810704FEAE77807EB1878C8F307188B
:1045900005F800801EE02C4FD7ED000A2B4F3F8816
:1045A00000EE107AB8EE400A60EE800A34F810701F
:1045B00000EE107AB8EE400A80EE801A244F97ED94
:1045C000000A31EE400ABCEEC00A10EE107A2F54F9
:1045D00000E000BF00BF471CB8B29042CDDB30E026
:1045E0000E462AE033B1012B23D134F8107026F89F
:1045F00010701FE0144FD7ED000A144F3F8800EEF3
:10460000107AB8EE400A60EE800A34F8107000EEBE
:10461000107AB8EE401A80EE810A0D4FD7ED000AED
:1046200030EE600ABCEEC00A10EE107A26F8107068
:1046300000E000BF00BF471CB8B29042D2DB00E0F0
:1046400000BF00BFBDE8F081D4000020CC000020F6
:10465000D0000020F0B504460D460020002113B123
:10466000012B5AD126E022E0266836F81060052E8C
:104670000BDD666836F81060294F3F887E43276857
:1046800037F81070B6FBF7F101E0264E3188254E61
:104690003688B14201D9234E3188234E3688B14243
:1046A00001D2214E318825F81010461CF0B29042FC
:1046B000DADB33E02EE0266836F810701B4E3688C1
:1046C000761FB74214DA666836F81060174F3F88D5
:1046D000BE1B134F3F887E43276837F81070DFF802
:1046E0004CC0BCF800C0ACEB0707B6FBF7F101E02B
:1046F0000C4E31880B4E3688B14201D9094E3188B3
:10470000094E3688B14201D2074E318825F8101083
:10471000461CF0B29042CEDB00E000BF00BFF0BD0F
:10472000CC000020C8000020CA000020CE000020DD
:1047300010B59DED020A214C2080214C2180214C96
:104740002280248800EE904AF8EE601A1C4C2488DF
:1047500000EE904AF8EE600A81EEA01A194C248807
:1047600000EE904AF8EE601A144C248800EE904A4D
:10477000F8EE600A81EEA02A71EE420AB8EE401A05
:10478000C1EE201A104CC4ED001A94ED001A0D4C25
:10479000248800EE904AF8EE600A21EE201A074CB9
:1047A000248800EE904AF8EE600AC1EE201A074C09
:1047B000C4ED001A064C238010BD0000C800002084
:1047C000CA000020CC000020D4000020D00000202F
:1047D000CE000020034610B50020024603E09C5C9A
:1047E000521C204480B28A42F9D310BD70B50546F0
:1047F0004FF6FF7000224AF201040EE0AB5C584015
:104800000023C60702D084EA500000E040085B1C89
:10481000DBB2082BF5D3521C92B28A42EED370BDA4
:104820002DE9F05F1D46DDE90A6ADDE90C9B1746BC
:104830008846040012D08421FBF740FDC4F80080B4
:10484000A780A56006B13546E560A4F810A0C4E9CC
:10485000059B2046BDE8F05F00F01BB8BDE8F09F67
:1048600010B54FF0FF3420B11AB190F86C300A2B1C
:1048700001D3204610BD00EBC303197790F86C10EC
:1048800000EBC1010A6210F86C1F491C0170002086
:1048900010BD002100F8781F4180818070472DE90C
:1048A000FC4194460400089A4FF0FF3034D065690B
:1048B000002D31D05D1DAEB2B51CAFB2258ABD4210
:1048C0002AD30AB1E56800E0A56845F6A520ADF851
:1048D00000008DF80210ADF80360009828609DF884
:1048E00004002871BCF1000F05D023B11A466146BF
:1048F000681DFBF7CAFC31462846FFF777FFADF885
:104900000000A819BDF800100180626902B03946A4
:104910002846BDE8F0411047BDE8FC81002800D0E2
:104920004167704710B504460078002806D0626AD7
:1049300012B10021A06990470020207010BDFEB583
:10494000040045D0022A43D30E468D1C921E0978DE
:10495000002790B2012916D0022939D121780029E7
:1049600036D0717894F801C0614531D102282FD337
:104970002988ADF800106189BDF80020914228D047
:10498000002261463BE0062822D32046FFF7CAFFFB
:10499000012121707078607028686060A88820818B
:1049A0006181FF20E7608DF8040070788DF80500C4
:1049B00046F66F30ADF80600208AADF80800606951
:1049C00001AA002804D000910623FB21FFF767FF0E
:1049D000FEBDA91C801E85B2012A06D0236AB3B190
:1049E0002A46A069984740B111E0E6697EB10A46BF
:1049F0002B466146A069B047F5E761780022204662
:104A000000F032F82046BDE8FE40FFF78BBFE068BB
:104A100001222844E0606089401C60816178204662
:104A200000F022F8608921898842D1D96168E06864
:104A3000626A884203D132B10121A06902E012B159
:104A40000021A06990472770FEBD2DE9F0411D4669
:104A500016460F46040005D02821FBF72FFC67619E
:104A60002682A561BDE8F0811CB500281BD04369F2
:104A7000002B18D002238DF804308DF8051022B1D8
:104A80006F218DF806106B2103E04E218DF8061082
:104A900047218DF80710012100914069042301AAE4
:104AA000FB21FFF7FCFE1CBD002802D01C3080E873
:104AB0000E00704710B538B131B10A4601460320E7
:104AC00001F0C4F9002010BD4FF0FF3010BD000010
:104AD00010B504460A464FF480610648FEF70EFC06
:104AE000002806D002462046BDE81040014901F0EA
:104AF000ADB910BDF02A00209321014800F074BD2B
:104B0000F02E002070B51D4B1B68C3F30224C4F1C6
:104B10000706042E00D90426231D072B01D20024EA
:104B200000E0E41E012303FA06F56D1E0D40A540CA
:104B300003FA04F1491E11400D43002807DB00BFB2
:104B400000F1E0214FEA051281F8002407E000F0AF
:104B50000F0202F1E0224FEA051182F8141D0BDB6F
:104B600000F01F014FEA50104FEA800000F1E020F2
:104B700003FA01F3C0F8003170BD00000CED00E055
:104B8000064900F0070208684FF6FF03184040EAA4
:104B90000220034A10430860704700000CED00E05B
:104BA0000000FA0530B504468078C1B00B4648B124
:104BB00001282AD1607801282FD0022832D003287A
:104BC00036D03DE00020ADF800016178684601294B
:104BD00002D0022905D01AE040A9801CFDF714FE7E
:104BE00003E040A9801CFDF7DBFD80B16F208DF84C
:104BF00000006B208DF80100BDF800016A46801CA2
:104C000083B22146022000F0CDFC41B030BD00222D
:104C10002146022000F0B4FCF7E711461846FDF7E4
:104C20004BFE03E011461846FDF70EFE054604E074
:104C3000FDF73CFD0546FDF71DFB0DB1012200E02F
:104C4000002241B02146BDE83040022000F098BC6F
:104C500010B504468078E4B000283ED15D905E90A7
:104C60005F9060906190629005A8FDF7CDFBB0B3B6
:104C7000DDF85D005D90DDF861005E90BDF86500D7
:104C8000ADF87C01DDF867006090DDF86B006190A5
:104C9000BDF86F00ADF888016F208DF874006B20AF
:104CA0008DF875000DF14E000DF14601CDE90110B2
:104CB0001938009060AA5DABCDE9033205AB0B4A11
:104CC000FE214130FCF73AFC002809DD801C83B24C
:104CD0001DAA2146022000F065FC64B010BDFFE76C
:104CE00000222146022000F04BFCF6E7C4600008D9
:104CF0004378012B0FD18378012B0CD1002A0AD0E5
:104D00000A7805490AB1012A00D10A700122014638
:104D1000022000F035BC7047BA0000202DE9F041B8
:104D200007460025C8680C462E46B0F57A7F5BD250
:104D3000401CE0602168A068095C5B2954D1401CDC
:104D4000A0602046FDF762FF4CB1D4E90110884213
:104D500003D22268125C5D2A33D0884203D3A06854
:104D6000401EA06040E0401E04F11008A0604046D4
:104D7000FDF7B4FF98B30DB3306046600646A068F7
:104D8000401CA0602046FDF741FF2146304600F060
:104D9000FFF930B32046FDF739FF14B3D4E9011011
:104DA000884203D22168095C2C29E0D062689042D5
:104DB00017D22168085C5D2813D102E005462E4613
:104DC000DDE7E068401EE06005B16E602020C7E9C5
:104DD0000250A068401CA0600120BDE8F081FFE700
:104DE00015B12846FDF72AFF0020F6E7034610B567
:104DF00000200246995CA1F13004092C01D830381A
:104E00000AE0A1F14104052C01D8373804E0A1F1F2
:104E10006104052C08D857380844032A00D2000141
:104E2000521C042AE6D310BD002010BD2DE9F04726
:104E30004FF000092DED028B82B007460C004FF0B9
:104E40002E0A48464D46C846CDF8009041D023680A
:104E5000DBB3D4E9012122E05E18865D342E1BD03D
:104E60000ADCA6F12B06092E1CD2DFE806F0151B82
:104E7000152F1B1515151500382E0DD006DC352EF7
:104E80000AD0362E08D0372E0CD105E0392E03D0AB
:104E9000452E01D0652E05D16D1C401C14B10E1895
:104EA0009642D9D32169681C8847060011D0A168B1
:104EB00020682A4601443046FBF7E7F906F80590DA
:104EC000B8F1000F13D000200FE002E04FF001080E
:104ED000E2E7002002B0BDEC028BBDE8F087315C58
:104EE0002E2901D106F800A0401CA842F7D369463C
:104EF0003046FCF77DFB0098B0EE408AF0EE608A09
:104F0000864203D1616930468847E2E79FED150B81
:104F100087ED068B53EC102B51EC180BFBF714FDAF
:104F200002D86FF000400FE09FED100B51EC180B12
:104F300053EC102BFBF7F0FC02D84FF0004003E0DD
:104F400051EC180BFBF7C9FC78610820F860009958
:104F5000A068891B0844A060616930468847012029
:104F6000B8E700000000C0FFFFFFDF4100000000C5
:104F70000000E0C12DE9F04107460026C8680C4654
:104F80003546B0F57A7F7BD2401CE060002C77D0AC
:104F9000D4E90110884273D22168095C7B296FD162
:104FA000401CA0602046FDF731FED4E90110884284
:104FB00003D22268125C7D2A4FD08842A0F1010002
:104FC000A0605DD204F110084046FDF787FEE8B30B
:104FD0000EB3286045600546CCB3D4E90110401CEF
:104FE00088424AD2A0602046FDF710FE214628469E
:104FF00000F048F858B32046FDF708FE28692862FB
:1050000000202861D4E90110884236D22168095C69
:105010003A2932D102E006463546DDE7401CA06061
:105020002046FDF7F3FD2146284600F0B1F870B1A7
:105030002046FDF7EBFDD4E90110884203D2216838
:10504000095C2C29C0D06268904201E014E014E0B1
:1050500013D22168085C7D280FD1E068401EE06013
:1050600006B175604020C7E90260A068401CA060DE
:105070000120BDE8F08103E016B13046FDF7DEFD0A
:105080000020F6E72DE9F84380468B6808684FF06A
:105090000009C418CDF8009008680E46651CC15C74
:1050A000641C22296ED10022716808E0BCF15C0FFB
:1050B00004D17F1C8F4265D2521C641C641C271AC9
:1050C0008F4204D294F800C0BCF1220FEED1271A0F
:1050D0008F4257D22178222954D11844201A801A9D
:1050E0003169401C884707004CD0009737E0297889
:1050F0005C2905D000986D1C00F8011B00902EE083
:105100000220611B012939DB6A78662A14D008DC89
:10511000222A12D02F2A10D05C2A0ED0622A2DD13A
:1051200008E06E2A0ED0722A0ED0742A0ED0752A8C
:1051300024D10DE0082200E00C22009901F8012B97
:1051400000910BE00A22F8E70D22F6E70922F4E7C6
:105150006A462146284600F0CDFE78B10544A542B6
:10516000C5D3009981F800901021C8E90317306871
:10517000201A401CB0600120BDE8F88317B17169A6
:105180003846884715B13068281AB0600020F3E728
:1051900070B50C0005465ED0206800285BD0A16881
:1051A00063680A1D9A4205D80844042231A1FBF71E
:1051B000BCF878B3A0686268411D0126914206D808
:1051C0002168052208442DA1FBF7AFF828B3A06899
:1051D0006268011D914206D821680422084429A171
:1051E000FBF7A3F8E8B1D4E90101814203D22268B8
:1051F000525C222A1DD0814221D22268525C2D2A83
:1052000002D0303A092A1AD821462846BDE8704013
:10521000FFF70CBE0420E86006E0EE60A068401DC9
:1052200004E002206E61E860A068001DA06001201B
:1052300070BD21462846BDE87040FFF723BF81427C
:1052400003D22268525C5B2A07D0814203D22068D5
:10525000405C7B2807D0002070BD21462846BDE871
:105260007040FFF75BBD21462846BDE87040FFF760
:1052700081BE00006E756C6C0000000066616C738E
:105280006500000074727565000000002DE9F041B2
:1052900004468078C2B00B46012804D161783F29CA
:1052A0001ED03D2923D061786D463F2904D023DCF0
:1052B00000297CD03D2917D188B3022814D1022AB5
:1052C0004BD31888ADF804018046FDF795F9BDF879
:1052D0000411491EC1EB01110E0186423DD24DE081
:1052E00011461846FDF7BAF942B0BDE8F081114603
:1052F0001846FDF797F9F7E76F266B274D2914D06D
:105300004F29F1D130B10128EED111461846FDF7F1
:10531000FBFB11E041A9A81CFDF7CAFB13E01EE04E
:105320002146AA2000F02CF9DEE740B10128DBD1AC
:1053300011461846FDF7DAFB78B10122F0E741A9E2
:10534000A81CFDF78DFB40B18DF800608DF8017051
:10535000BDF80401801C83B222E00022E0E7FDF7E3
:105360004BF9F02200F1EF01B1FBF2F1ADF80411BD
:10537000009088B2ADF80400062311E0F02706F192
:10538000F001814201D9801B87B2ADF80080FDF7A2
:105390002FF981193A46A81CFAF777FFBF1CBBB258
:1053A0006A462146AA2000F0FDF89DE7FFE70128A4
:1053B0009AD1FDF727FB20B1FDF706F908B10122CC
:1053C00000E000222146AA2000F0DAF8FCF752FFA4
:1053D0008AE70000F0B50446807899B015460E467D
:1053E00001281FD1607802281ED001281AD15DB390
:1053F000112D29D26846FDF707F828B30DF12100D9
:1054000011210746FAF75AFF2A4631463846FAF77D
:105410003CFF6846FDF7B2F8B0B101222146AA2050
:1054200000F0AEF819B0F0BD002AFBD008780128D2
:1054300000D000200549087019B02146BDE8F040B1
:105440000122AA2000F09CB80022E7E7BB00002060
:1054500010B501214FF44010FEF766F8012107480E
:10546000FEF762F801210648FEF75EF803480121C5
:10547000BDE810401530FEF757B8000001003000BD
:105480000800440010B50A49094A0A4C0B681C324E
:10549000A34209D112684FEA33239A4204D1202251
:1054A000FAF7F3FE012010BD4FF0FF3010BD0000F1
:1054B000001001085AA55AA52DE9F04704008A46B4
:1054C00016D054F8047CD4F800903E1F564500D9FD
:1054D00056462046FCF75CF805468846324621468B
:1054E0005046FEF7D5FF40B1C0F80090BDE8F08708
:1054F000BDE8F0470846FCF78FB844E9017955B19B
:1055000029686A18211F8A4202D9611B091F296074
:10551000C5F80480EAE7024AC2F80080E6E7000026
:10552000D80000201CB501214FF44010FDF7FCFF0E
:105530006846FEF773FD01208DF8070000218DF805
:1055400004108DF806000820064C00908DF8051018
:1055500069462046FEF76CFD08212046FEF7F8FC60
:105560001CBD00000000024003484078192802D307
:105570000248FBF7BFBD7047080000203C07002031
:1055800008B522B16F228DF800206B2203E04E2275
:105590008DF8002047228DF8012002236A4600F092
:1055A00001F808BD38B51C4613000D4A05460878B9
:1055B0001070487850708878907006D02CB10848E8
:1055C00022461946C01CFAF760FE002000900548EC
:1055D000E41CA3B2024A29464068FFF760F938BDCF
:1055E00018300020B00000207CB50C460546FEF7C0
:1055F000CBFC21462846FEF7A3F801211148FDF710
:1056000093FF684600F022F800208DF800008DF826
:10561000010005218DF802100B4C8DF8030001905C
:105620006946204600F02CF80121204600F023F8BE
:105630000121204600F01AF80121204600F011F85F
:105640007CBD00000C0044000030014000210170CE
:1056500041708170C1700171417181710121C1710D
:105660007047026861F3861202607047426861F316
:10567000000242607047426861F341024260704735
:10568000C26922F40062C2610A7832B1012A08D0EC
:10569000022A12D0032A18D023E0026822F4004222
:1056A0000EE0026822F400420260026822F48042A6
:1056B0000260026842F4806212E0026842F4004232
:1056C0000260026822F4804206E0026842F400426E
:1056D0000260026842F480420260026822F4806242
:1056E0000260CB79026863F3492202604A78012A9A
:1056F00002D1CA79012A18D0026822F480720260AD
:105700004B78026863F3820202608A78072A10D815
:10571000426822F400724260426822F48072426061
:105720008B78026863F3C50231E0026842F480724C
:10573000E5E70A2A426820D022F4007242604268FB
:1057400042F4807242608A78036862F3C5030360A2
:10575000CB78026863F3C71202600B79026863F3C7
:10576000CB2202604B79026863F3410202608A79BE
:10577000016862F300010160704742F40072426008
:10578000426822F480724260026822F038020260AD
:10579000DEE7000010B5FDF7F9FE1D4940F2531099
:1057A000086001211B48FDF7BFFE1B48016921F07D
:1057B0000301891C016101210846FDF705FE00BFB8
:1057C000FDF79EFE0028FBD001231A464B21184608
:1057D000FDF7C0FE01210220FDF7F6FD1920FDF7BF
:1057E0007DFE0128FAD10020FDF7BEFD0020FDF767
:1057F000D5FD0020FDF7CAFD0220FDF703FF00BF25
:10580000FDF712FF0228FBD1BDE8104000F006B8FA
:10581000003C02401C0040000070004070B5FDF7E5
:1058200003FF2249224A234C20B101281FD002281D
:1058300011D120E01E48001F03685B0405D50068F5
:10584000C00402D51C48206000E021601068216877
:10585000C0F30240C140216015489C3800681749D8
:10586000C0F30310085C2168C140216070BD10685E
:10587000C0F3C240EEE70E48A0380268036805682E
:10588000C3F38813006805F00F050C4EC0F3024007
:10589000B61F305C15FB00F2A1FB03010023FAF7F1
:1058A000BDFC49084FEA30002060D5E700127A00BD
:1058B000A438024034000020006CDC02DE5F0008E7
:1058C00070B50E484FF47A710068B0FBF1F0401EDD
:1058D000B0F1807F11D24FF0E024606165170F2195
:1058E0002846FBF745FE0020A061072020612846DE
:1058F000BDE870400021FBF73BBEFEE7340000200E
:10590000C1628262416941F00101416170470268F0
:1059100061F3061202607047026861F300020260E0
:105920007047C943016170470246002012690A426C
:1059300000D001207047012A05D0002A02D1C26898
:105940008A43C2607047C2680A43FAE72DE9F04112
:105950000F4D14460E462878002816D0FCF748FE56
:105960000746FCF749FE3918686888420CD20219CC
:105970008A4201D9091A8CB234B122463146FAF76B
:1059800084FC6868204468600120BDE8F081000064
:105990004034002070B50F4C2078B0B1A9B1FCF7AD
:1059A0002BFE0546FCF724FE6168091AA9420CD3B8
:1059B000207AAA2809D1607A3D2806D1FCF718FE82
:1059C000A9B2FCF72FFEFCF75DFC002020706060A0
:1059D00070BD0000403400202DE9F0411E46144601
:1059E000AA290CD1032E0AD32078032807D1A07846
:1059F000012804D160783F2804D03D2802D000203F
:105A0000BDE8F0810F4D01222A7068722972FCF7FF
:105A1000EFFDF61EB6B26860FCF7EAFD0746FCF73C
:105A2000EBFD3918686882198A4201D9091A8EB2C9
:105A300036B1E11C3246FAF728FC686830446860E9
:105A40000120DDE7403400202DE9F047814688B091
:105A500001216048FDF768FD01215F48FDF764FD05
:105A60005C4801211530FDF75FFD05A8FEF7D6FA69
:105A700001258DF81B5000248DF818400227DFF80F
:105A80005C818DF81A70AE0205968DF8194005A953
:105A90004046FEF7CDFA07220A214046FEF7FAFA01
:105AA0008DF81B508DF81840E8028DF81A7005909B
:105AB0008DF8194005A94046FEF7BAFA07220B21D6
:105AC0004046FEF7E7FADFF818A100231A464946D8
:105AD000504600F0CFF80121504600F0B1F9012105
:105AE000504600F0A8F90121504600F0A5F8002228
:105AF00002212720FFF706F801223A49504600F01C
:105B00002DF9DFF8E4804046FDF7DEFE6846FDF73C
:105B10008CFEADF80A601020ADF808008DF80F403B
:105B200032488DF80D5001900AF104078DF80E40AF
:105B30008DF8115000978DF80C408DF81040694693
:105B40004046FDF78FFE0121504600F070F8DFF867
:105B500098800121A8F158084046FDF7E3FE22484D
:105B60001D21BC30FDF7E5FEDFF87C9009F114093A
:105B70004846FDF7A9FE6846FDF757FE8DF80F4031
:105B80001B488DF80D50ADF80A6001908DF80E405D
:105B90008DF81150ADF8084000978DF80C408DF845
:105BA000104069464846FDF75DFE0121504600F071
:105BB00039F801214846FDF77DFD01214046FDF7FA
:105BC000B1FE09481C21C030FDF7B3FE08B0BDE8A6
:105BD000F087000001003000120040000004024085
:105BE0000048004004000C0058600240C80A002031
:105BF000C80E002010B5FFF727FF07494FF4806457
:105C00002246A1F50860FBF709FA2246BDE81040DC
:105C100002490348FBF702BAC8120020C81A002044
:105C2000980A0020426961F3861242617047426916
:105C300061F3C71242617047C26861F34D32C260BE
:105C400070474FF40062914205D09201914202D018
:105C5000D200914201D102627047CA0602D00168A7
:105C600040687047C943016070470068084000D031
:105C7000012070472DE9FF5F04469B4691468A4606
:105C80006846FDF7C3FB2E482E4FDFF8BC802F4E31
:105C90004FF4004584420ED10020FDF7CDFCE0B169
:105CA000012815D003281BD0D8F800003D46C004B9
:105CB00016D5354614E02648844201D1012003E080
:105CC0002448844206D10220FDF7B6FC38B1E7E74C
:105CD000009D05E02048844201D1029D00E0039D23
:105CE00005EB85004100B1FBFAF00A21B0FBF1F2AF
:105CF00001FB1202B0FBF1F0052A00D3401CA168A1
:105D000060F30F01A160B9F1020F10D0E068B9F1A2
:105D1000000F20F080500DD0E060E06840F480502B
:105D2000E06021696BF30D312161BDE8FF9FE06800
:105D300040F08050E060E06820F48050F0E7000020
:105D40000010014000127A00A0380240006CDC0212
:105D500000440040004800400014014010B501F02C
:105D60001F0400EB11400123A3400168012A02D067
:105D70009943016010BD1943FBE740292DD00EDC8B
:105D8000082932D006DC01293ED0022938D0042966
:105D90004FD135E010292FD020294AD121E0B1F58B
:105DA000006F35D008DC802913D0B1F5807F0ED08C
:105DB000B1F5007F3DD106E0B1F5003F2CD0B1F543
:105DC000801F36D12CE04269C2F380222BE00269A9
:105DD00004E0C268C2F3C01225E0C268C2F38012B8
:105DE00021E0C268C2F340121DE0C26892061BD4D3
:105DF0004269D20718D11CE0C268C2F3001212E057
:105E0000426902F001020EE0C268C2F300220AE019
:105E1000C268C2F3806206E0C268C2F3803202E068
:105E20004269C2F3403222B10068084000D001202C
:105E3000704700207047C26861F38202C2607047F9
:105E4000C26861F3C302C2607047000070B5224DA2
:105E500006283ED2DFE800F03D030D1A25301F482A
:105E6000FBF717F90404240C31D0012229461C4801
:105E700009E01A481030FBF70CF90404240C26D072
:105E8000012229461748FFF769FF20E01348203018
:105E9000FBF7FFF80404240C19D00122294612480C
:105EA000F1E70E483030FBF7F4F80404240C0ED070
:105EB000012229460D48E6E708484030FBF7E9F89B
:105EC0000404240C03D0012229460948DBE7E0B290
:105ED00070BD002070BD000006000C00780A002094
:105EE000001001400044004000480040004C0040C9
:105EF000005000402DE9F04705460027481B164694
:105F0000894606285DDBA81CFEF770FF0446A0F555
:105F10005C414FF48060814253D3A4F558418246DE
:105F200051451AD2A81DA9EB00014FF00C08062913
:105F300047DB01785C2944D14178752941D1801C27
:105F4000FEF754FFA0F55C4151453AD2C4F3090174
:105F500061F39F2000F5803002E04FF006082046F4
:105F6000802801D2012110E0B0F5006F02D2022199
:105F7000C0270AE0B0F5803F02D20321E02704E009
:105F8000B0F5881F1DD20421F0274A1E08E000BF8B
:105F900000F0BF03346843F080038009A354521E0D
:105FA00012F0FF02F4D1012901D9384301E000F0D9
:105FB0007F00326810703068084430604046BDE8A9
:105FC000F0870020FBE700003D3D00089D3D0008F4
:105FD0003D390008852B000801020408102000004C
:105FE0000000000000000102030406070809010286
:105FF000040810200000000001020304000000005B
:10600000010203040000000000000000010203047C
:106010000607080901000000F14C00083F000000DD
:10602000514C00083D000000A54B00080100000095
:10603000D5530008030000008D5200080040404086
:10604000404040404040414141414140404040404B
:1060500040404040404040404040404040050202F7
:1060600002020202020202020202020202202020B6
:106070002020202020202002020202020202909012
:106080009090909010101010101010101010101010
:106090001010101010101010020202020202888864
:1060A0008888888808080808080808080808080870
:1060B0000808080808080808020202024000000058
:1060C0003D6000087B22504E223A222573222C226A
:1060D000534E223A222573222C225356223A22254D
:1060E00073222C22485649223A222573222C225808
:1060F00059223A222573222C2250726F746F636FDB
:106100006C223A222573227D000000002C610008D9
:1061100000000020E0000000681600080C62000883
:10612000E0000020B04A00007816000800000000DF
:10613000000000000000000000000000000000005F
:10614000000000000000000000000000000000004F
:106150000000000007060504030201000F0E0D0CED
:1061600000127A00000000000000000080008000A3
:1061700080000000000402400004024000040240CD
:10618000010030000100300001003000000000007C
:1061900000000000000000000000000000000000FF
:1061A00000000000000000000000000000000000EF
:1061B000000000001916000891150008B9540008E5
:1061C00000000000000000000000000000000000CF
:1061D00000000000000000000000000002000000BD
:1061E0000000000000000101000514000000000094
:1061F00000000000B80B14006400FF0F0000000056
:0C62000000000000000000000000000092
:04000005080001E10D
:00000001FF
